:020000040000FA
:06000000052817000700AF
:08000800152883128501073061
:10001000990083169F01EF3085000730950040302E
:10002000810083122620051655201628000009306D
:1000300057205F200512593057205F205520851921
:1000400013282620051690308B002528A3010518BB
:1000500023148518A3140800F13EA00020183028AE
:10006000A0183228A0183428FC3E031834280800B1
:10007000FF3EA1005E302C2060302C20A10B3C28DC
:100080000800FF3EA200633038205D302C20633032
:1000900038205F302C20A20B472808005220532024
:1000A0005320522053205620000000000800A400D6
:1000B0005A28542000005F20A40B59280800230868
:1000C0000339820766286A286E287228183038207B
:1000D00050302C283E3038201E302C287C303820E0
:0C00E00050302C28F930382050302C28EB
:02400E00C33FAE
:00000001FF
